:020000040000FA
:0400000000008B2849
:080008008C105F080319142895
:10001000DF1C0E2805187828DF100900051C6E2843
:10002000D001D101D201DF0150085302D6000318DC
:10003000322851085402D700031821280130D70272
:1000400025280130D7020318372852085502D80056
:1000500003182D280130D80266280130D802031C6D
:1000600066283D2851085402D700031C2528520851
:100070005502D800031C66283D2853085002D600BC
:1000800003185B2854085102D70003184A2801308E
:10009000D7024E280130D7020318602855085202B3
:1000A000D800031856280130D80270280130D80231
:1000B000031C7028090054085102D700031C4E2865
:1000C00055085202D800031C702809000130D002E4
:1000D00003186E28D10203186E28D202E003792893
:1000E0000130D007031C7828D107031C7828D207D9
:1000F000E00A600807397E2086000900DE00003033
:100100008A005E0882078034A03420346034403492
:10011000503410349034D001D101D201D301D40134
:10012000D5010330DF004130C000BD01C101C20173
:10013000C301C401C501C601C701C801DB012030EC
:10014000B8008312B901380884003908840783167F
:100150009B001C141A0883128000B90A0F30390260
:10016000031DA3285A30B200B300B4003930B500E3
:10017000B6003230B000B1012930B800B901BA017F
:10018000BB01BD0107309F0083160F308600FF3092
:10019000850083128316BE30920083120F309200C6
:1001A00083164D30990020309800831290309800CB
:1001B0008B170B1783168C1483128B178C1AE3285A
:1001C000DB1BAB29DE288B131A08BC008C123B18F2
:1001D0003C29BA1B12293008840031088407000822
:1001E0003C02031DFD28B10A05303102031DFE2823
:1001F000B101B901FF30BA00DD28B101380884002F
:100200003908840700083C02031D1029B90A05308B
:100210003902031DDD28B101B901FF30BA00DD2824
:10022000B901DD283C08BA00FF30BB0001308A006C
:100230003A080F392721CD004D0803194A29BD017D
:10024000DD01CD1FDD28CD132808DD00DD28DE000F
:1002500001308A005E08820700340334833400349E
:1002600000340034003400340034053401340034E8
:100270000034003400340034DD0803194129DD0363
:10028000DD28400884003D0884073C088000BD0A42
:10029000CD0BDD28BD01BB0101308A003A080F39C2
:1002A000543E03188A0A82008B28642964298B280B
:1002B0008B288B288B288B286B297D2973298B28E9
:1002C0008B288B288B288B284108D3004208D40028
:1002D0004308D500DD280830DA001130DC00813019
:1002E000DB00BA01DD284108A8000830DA00283018
:1002F000D9000130BE00BA018E294108A900420888
:10030000AA004308AB004408AC004508AD00093022
:10031000DA002930D9000530BE00BA01590884003E
:10032000000883169A0083125A0883169B009C11BA
:100330001C1555309D00AA309D009C141C11831281
:100340008C1FA0298C13DA0AD90ABE0B8E29B90199
:10035000BA01BB01DD288B130C1EDD285A08831659
:100360009B001C141A0883129900DA0ADC0BDD28A2
:04037000DB01DD28A8
:02400E00613F10
:1042000000000000000000000000000000000000AE
:10421000000041004C0054003000310020004100FB
:104220005200430052002000560031002E003000A2
:04423000300030002A
:00000001FF
